:100000000C940F030C9447030C9447030C94470380
:100010000C9447030C9447030C9447030C94470338
:100020000C9447030C9447030C94AE260C94802741
:100030000C94A2210C9447030C9447030C9447039F
:100040000C9447030C9447030C9447030C94470308
:100050000C9447030C942A220C9447030C944703F6
:100060000C9447030C9447030C9447030C944703E8
:100070000C9447030C9447030C9447030C944703D8
:100080000C9447030C9447030C9447030C944703C8
:100090000C9447030C9447030C9447030C944703B8
:1000A0000C9447030C9447030C944703CB06CB06F0
:1000B000F706F7065F077D0795089508880721086A
:1000C00032083208ED2714280C2914280C2960283E
:1000D00083280C29DA28E928A8002900000000005C
:1000E00000000000000000000000000031002D00B2
:1000F0002E004A002B0014001A00080015001700FB
:100100001C0018000C00120013002A004B00E00035
:1001100004001600070009000A000B000D000E0085
:100120000F00330034004E00E1001D001B000600EC
:1001300019000500110010003600370038002800B3
:100140004D004C00E300E200035101512C002C0053
:1001500002515000510052004F0001000100000008
:1001600000000000000000000000000000002F0060
:1001700030003500AE0001001E001F0020002100ED
:100180002200230024002500260027000100AB00E8
:1001900001001E021F022002210222022302240269
:1001A0002502260227023402AC00010001000100F2
:1001B0000100010001000100010001000100010037
:1001C0000100AD000100010001000100010001007B
:1001D00001000100010001000100010046000100D2
:1001E000000000000000000000000000000000000F
:1001F0002F02300235020100010001000100010060
:1002000001000100010001000100010001000100E6
:10021000010039000100010001000100010001009E
:1002200001000100010001000100010001000100C6
:1002300001000100010001000100010001000100B6
:1002400001000100010001000100010001000100A6
:100250000100010001000100010001000100005740
:10026000C35C00000000000000000000000000006F
:100270000000440045006800010001003A003B0016
:100280003C003D003E003F00400041004200430072
:100290000100010001000100010001000100010056
:1002A0000100010001000100010001000100010046
:1002B0000100010001000100010001000100010036
:1002C0000100010001000100010001000100010026
:1002D0000100010001000100010001000100010016
:1002E0001E140A052223252628292A2C2D2F3032D8
:1002F000333536383A3B3D3E4042434547494A4C08
:100300004E5051535557595A5C5E60626466686935
:100310006B6D6F71737577797B7D7F81838587893D
:100320008A8C8E90929496989A9C9E9FA1A3A5A742
:10033000A8AAACAEAFB1B3B4B6B8B9BBBCBEBFC16E
:10034000C2C3C5C6C7C9CACBCCCDCED0D1D2D2D3F9
:10035000D4D5D6D7D7D8D9D9DADADBDBDBDCDCDC0D
:10036000DCDCDDDDDDDDDCDCDCDCDCDBDBDBDADAD0
:10037000D9D9D8D7D7D6D5D4D3D2D2D1D0CECDCC47
:10038000CBCAC9C7C6C5C3C2C1BFBEBCBBB9B8B65C
:10039000B4B3B1AFAEACAAA8A7A5A3A19F9E9C9AE7
:1003A00098969492908E8C8A89878583817F7D7BB5
:1003B00079777573716F6D6B6968666462605E5C96
:1003C0005A5957555351504E4C4A4947454342405C
:1003D0003E3D3B3A3836353332302F2D2C2A2928F2
:1003E0002625232200010101010101010101020270
:1003F00002020202020202030303030303030304D3
:10040000040404040404050505050506060606069D
:10041000070707070708080808090909090A0A0A57
:100420000B0B0B0C0C0C0D0D0D0E0E0E0F0F0F10F9
:100430001011111112121313141415151616171783
:10044000181819191A1A1B1B1C1D1D1E1E1F2020EF
:10045000212222232424252626272829292A2B2C39
:100460002D2D2E2F30313232333435363738393A5C
:100470003B3C3D3E3F404142434445464748494A54
:100480004C4D4E4F50515354555658595A5B5D5E22
:100490005F616264656668696B6C6D6F70727375BD
:1004A00077787A7B7D7E8082838587888A8C8E8F21
:1004B00091939596989A9C9EA0A2A3A5A7A9ABAD4F
:1004C000AFB1B3B5B7BABCBEC0C2C4C6C9CBCDCF3D
:1004D000D1D4D6D8DBDDDFE2E4E7E9EBEEF0F3F5EB
:1004E000F8FAFDFF12035400680065002000410087
:1004F000760065002E00000018034B0069006E00B6
:1005000067006C0079002D004B00650079007300D6
:1005100000000403090409023B00020100A0FA09DB
:100520000400000103010100092111010001224022
:100530000007058103080001090401000103000010
:1005400000092111010001227B0007058203200020
:100550000112010002000000084B4B25121100019E
:1005600002000105010902A10185020901A100059E
:100570000919012908150025019508750181020551
:1005800001093009311581257F9502750881060919
:10059000381581257F950175088106050C0A3802FA
:1005A0001581257F950175088106C0C00501098068
:1005B000A101850319012AB700150126B70095018D
:1005C00075108100C0050C0901A101850419012ADB
:1005D000A002150126A002950175108100C0050139
:1005E0000906A101050719E029E71500250195086D
:1005F000750181029501750881010507190029FF20
:10060000150026FF009506750881000508190129C7
:1006100005950575019102950175039101C011249D
:100620001FBECFEFDAE0DEBFCDBF04B603FE18C0B9
:100630008091DF029091E002A091E102B091E2028C
:100640008730904BA740B04B59F41092DF021092C4
:10065000E0021092E1021092E202E0E0F8E3099574
:1006600011E0A0E0B1E0E4EAF3E502C005900D92EC
:10067000AA3DB107D9F722E0AAEDB1E001C01D9271
:10068000AF3DB207E1F70E9493150C94D0290C946A
:100690000000CF93DF93FC012081223040F0EC0179
:1006A0000E946204CE01DF91CF910C94521FDF9122
:1006B000CF9108958130974519F088EC90E0089526
:1006C0008BEE90E00895811107C0662311F089EA4E
:1006D00001C08AEA0E94790681E0089561E080E025
:1006E0000E94BE1844E66FEF82E30E94621A82E025
:1006F0000E94FA1A2BEC32E040E069EB81EE0E9496
:10070000E0180C945619CF92DF92EF92FF92CF939C
:100710006B017C0141E00E94D609C82FC19543E0DE
:10072000C701B6010E94D609882311F088EC01C0E8
:1007300080E02BEC32E04C2F60E00E94E0180E9439
:100740005619C701B601CF91FF90EF90DF90CF907F
:1007500008959C013A9521153F4130F5BC0166276B
:100760007270AC01442754709C012227387094FFAA
:100770000FC090FF02C080E101C080E0672B09F04C
:100780008062452B09F08064232B79F080680895FE
:10079000892F8170672B09F08260452B09F08460F6
:1007A000232B19F08860089580E00895CF93DF939C
:1007B000EB010E94A903FE01DF91CF910994CF9331
:1007C000DF93EC01805E9109089710F0209719F4EF
:1007D00062E876E002C06DE079E0CE010E94D603C7
:1007E0008C2FDF91CF910C945005CF93DF93EC01C8
:1007F0000E94FA05CE01805E9109089710F02097BB
:1008000019F469E876E002C064E179E0CE01DF9195
:10081000CF910C94D60381E0089581E008950C9463
:100820000D0408950C9411041F93CF93DF9300D00F
:1008300000D01F92CDB7DEB749835A836B833091C6
:10084000DD0189819A81311114C0662359F0222378
:1008500049F00E94F50A182F682F89819A810E9419
:100860009E0A03C00E94C90A182F69817A81812FCC
:1008700004C00E94F50A69817A810F900F900F9051
:100880000F900F90DF91CF911F910C94FE12FC01FD
:10089000262F408151816281738184810C941404DC
:1008A00081E00895CF93DF93EC0160E00E9447045C
:1008B000BE01DF91CF910C9412040C9444140C945B
:1008C000401408950E9433090E9461042FEF84E3CD
:1008D0009CE0215080409040E1F700C000000C9463
:1008E00050220F931F93CF93DF938C0161E00E94FE
:1008F0004704EC01B8010E94991FB801CE010E9483
:100900000F04882309F44BC0B801CE010E94E41FF4
:10091000882309F444C0B801CE010E94B41E882384
:10092000F1F1B801CE010E943A1C8823C1F1B8014F
:10093000CE010E94EB1D882391F1B801CE010E94E7
:10094000911B882361F1F8018281882309F1CB355D
:100950008DE5D807C1F050F4C115FCE5DF0781F043
:10096000CF3DDC45A9F40E94E11019C0CC35EDE57E
:10097000DE0761F0CD35DD4559F40E94241008C032
:100980000E9462040CC00E942D1002C00E94301010
:10099000C801DF91CF911F910F910C940B0480E05F
:1009A000DF91CF911F910F9108950E9484210C94A3
:1009B000EE040E94F1040C948A2108950C94DD0445
:1009C00081E008950C94E0040895CF93C82F0E940D
:1009D000DE048C2F0E94E204CF91089580E00C94F5
:1009E000E5040E94C9200C94E5040E94C92090915E
:1009F000DC01891721F08093DC010C94E504089553
:100A0000CF93DF93CDB7DEB72B970FB6F894DEBF49
:100A10000FBECDBF4F83588769877A878B87611157
:100A20000E94700F9E012F5F3F4F86E0F9011192E7
:100A30008A95E9F785E0FE013796D90101900D927C
:100A40008A95E1F789819A814C815D81452B31F04E
:100A50009F3F31F491E08F3F19F403C091E001C052
:100A600090E090FF09C049815A816B817C818D8122
:100A70009E810E948E0E05C0C9010E945004811102
:100A8000F2CF2B960FB6F894DEBF0FBECDBFDF912D
:100A9000CF910895FC01808191810E94370B0895C8
:100AA000CF93882309F4A4C0C82F8238C1F40E94D0
:100AB000C92081FD9DC069E3809130019091310191
:100AC0000E945C210E94920F2FEF81EE94E0215052
:100AD00080409040E1F700C0000069E319C083380E
:100AE00001F50E94C92080FD83C063E5809130013B
:100AF000909131010E945C210E94920F2FEF81EEB4
:100B000094E0215080409040E1F700C0000063E590
:100B100080913001909131010E945E21CF910C941F
:100B2000920F8438C1F40E94C92082FD61C067E43D
:100B300080913001909131010E945C210E94920FBE
:100B40002FEF81EE94E0215080409040E1F700C00B
:100B5000000067E4DDCF8CEF8C0F813AD0F46C2F6E
:100B600080913001909131010E942621882349F023
:100B70006C2F80913001909131010E945E210E9482
:100B8000920F6C2F80913001909131010E945C2175
:100B9000C5CF80E28C0F883048F4C77081E001C077
:100BA000880FCA95EAF70E94500FB8CFEBE5EC0F1B
:100BB000E33040F4F0E0E358FE4F808190E0CF91C5
:100BC0000C94EE20E8E5EC0FE73150F4F0E0EE0F86
:100BD000FF1FE15BFE4F80819181CF910C94042136
:100BE000CD3E30F08C2F0E941816CF910C94EA164F
:100BF000CF910895882309F464C0823879F40E9463
:100C0000C92081FF5EC069E380913001909131017C
:100C10000E945C210E94920F69E310C08338B1F4F6
:100C20000E94C92080FF4DC063E580913001909102
:100C300031010E945C210E94920F63E58091300196
:100C4000909131010E945E210C94920F843879F4C6
:100C50000E94C92082FF35C067E4809130019091E5
:100C600031010E945C210E94920F67E4E7CF9CEF64
:100C7000980F913A10F4682FE1CF90E2980F9830D6
:100C800050F4877091E001C0990F8A95EAF7892F97
:100C90000E94560FD9CF9BE5980F933020F480E047
:100CA00090E00C94EE2098E5980F973120F480E0C6
:100CB00090E00C9404218D3E20F00E9473160C9459
:100CC000EA1608951F93CF93DF93182FEB010E942C
:100CD0005005209741F08FE99FE00197F1F700C0A0
:100CE00000002197F6CF812FDF91CF911F910C94B7
:100CF000FA05893319F060E070E002C060E570E049
:100D00000C946206882321F00E94500F0C94920FDD
:100D10000895882321F00E94560F0C94920F089595
:100D2000CF92DF92EF92FF920F931F93CF93DF93B7
:100D30007C01D62FC72FFC011281058102950F700F
:100D40000E94460F8823B9F01123A9F08C2F807FD1
:100D5000803421F080E28D0F883068F08091AE02FF
:100D600082FD09C082E00E94F20F0E94460F91E0CE
:100D7000D82ED92601C0D12CCC2EC2948FE0C82207
:100D80008C2D90E08C30910508F0CFC1FC01EA5A1F
:100D9000FF4F0C9468298C2F807FCF70882311F02F
:100DA000C295C07F112399F0CC2309F4AAC180E237
:100DB0008D0F883010F0D11104C08C2F0E94500F7D
:100DC00003C08C2F0E94630F0E94920F9AC18D2F37
:100DD0000E94FA05CC2309F4A8C180E28D0F883067
:100DE00038F1DD2329F18C2F0E94690F24C08C2F4C
:100DF000807FCF70803211F0C295C07FDD2319F063
:100E0000D130A1F13DC08091AE0282FF17C0112305
:100E100049F0CC2329F08C2F0E94500F0E94920F92
:100E200080E070C180E00E94FA05CC2309F47DC106
:100E30008C2F0E94560F0E94920F77C1112371F0E0
:100E4000002341F0013031F40E94730F8C2B0E947B
:100E50007B0F6BC10E94730F8C2B1DC0002319F0F8
:100E6000013009F462C10E94880F25C0112321F0CE
:100E7000063008F05AC10EC0053008F056C11BC03C
:100E8000112361F0002331F0F701858180FF39C122
:100E90008F7085838C2F0E94820647C1002359F0F2
:100EA000D93309F03FC1FFEF07EE13E0F1500040E6
:100EB0001040E1F735C18C2F0E94890636C18C2F76
:100EC00086958695837019F0813061F02EC11123CB
:100ED00021F08D2F9C2F937002C080E090E00E9443
:100EE000EE202BC1112321F08D2F9C2F937002C077
:100EF00080E090E00E94042120C18D2F112319F081
:100F00000E94181602C00E9473160E94EA1615C1AC
:100F10008C2F837009F047C011110BC12D2F229522
:100F200026952770220F220F6D2F6F70862F90E06D
:100F3000A0E0B0E0022E04C0880F991FAA1FBB1FBB
:100F40000A94D2F7D4FF10C04FE050E060E070E0A8
:100F500004C0440F551F661F771F2A95D2F740958E
:100F600050956095709503C040E050E0BA01C69579
:100F7000C695C3708A019B01082B192B2A2B3B2B8A
:100F8000C901B801C23049F058F4C13019F00E94CB
:100F90009F09CFC00E948D09CCC00E94B109C9C071
:100FA0000E948B09C6C0112319F08C2F817001C0DB
:100FB0008695882309F4BDC02D2F2295269527708C
:100FC000220F220F6D2F6F70862F90E0A0E0B0E00F
:100FD000022E04C0880F991FAA1FBB1F0A94D2F7C4
:100FE000D4FF10C04FE050E060E070E004C0440F58
:100FF000551F661F771F2A95D2F74095509560952B
:10100000709503C040E050E0BA01C695C695C37024
:101010008A019B01082B192B2A2B3B2BC901B801F4
:10102000C23049F058F4C13019F00E94790A81C0E9
:101030000E94670A7EC00E948B0A7BC00E94C5097D
:1010400078C0CF70112339F08C2F0E94000A8D2FA9
:101050000E9482066EC08D2F0E9489068C2F0E94EE
:10106000210A67C0D23F21F128F4D03F41F0D13F9F
:10107000C1F043C0D33F19F1D43F79F03EC01123F2
:1010800041F0053008F051C08C2F8F710E94460A44
:101090004CC0063008F049C0F7CF8091AE0282FF05
:1010A00018C0112339F08C2F8F710E94000A3DC0A7
:1010B0001123C9F38C2F8F710E94210A36C011238E
:1010C00029F08C2F8F710E94EB092FC00E94D1094B
:1010D0002CC0112349F0CF718C2F0E94000A63E0CD
:1010E0008C2F0E94D70F21C081E00E94F20F0230A6
:1010F000E0F082E00E94F20F18C0112331F00023CB
:1011000091F28D2F0E94500510C0002399F2D9331F
:1011100049F41FEF27EE33E0115020403040E1F753
:1011200000C000008D2F0E94FA0588EF8C0D8430DE
:1011300020F40E94C9200E94E504DD20C9F00E942D
:10114000420F80FD15C0F70112820E943C0F0E94E1
:10115000000AC7010E94D9080E943C0FDF91CF917D
:101160001F910F91FF90EF90DF90CF900C94210A88
:10117000DF91CF911F910F91FF90EF90DF90CF9073
:1011800008950F931F93CF93DF93EC0168817981CA
:101190008A810E94420B8C010E949D0A0E9479095B
:1011A000B801CE010E949006DF91CF911F910F915F
:1011B0000895CF93DF93EC01988189812B813C8145
:1011C000232B31F08F3F31F481E09F3F19F403C0AE
:1011D00081E001C080E080FD1DC0CE010E9471044D
:1011E000811110C00E94460F8823A1F08A818823B4
:1011F00089F08091AE0282FD0DC082E0DF91CF9137
:101200000C94F20FCE010E94C108CE01DF91CF9164
:101210000C945204DF91CF910895882321F00E940D
:10122000630F0C94920F0895882321F00E94690F98
:101230000C94920F089580E090E00E94EE2080E0F0
:1012400090E00E9404210E94700F0E94920F0E9461
:101250001B180C94EA1680913001909131010E9484
:1012600060210C941B090E945D0F0C942B09929530
:101270009F70963079F010F4925001C09A509230DD
:1012800068F4803F69F018F4883E40F409C0843F58
:1012900029F406C0883E20F0813F11F080E00895D7
:1012A00081E00895FC01808191810E94370B0E94AA
:1012B00037090895CF93DF9300D000D01F92CDB7A8
:1012C000DEB70F900F900F900F900F90DF91CF919E
:1012D0000895CF93DF9300D000D000D0CDB7DEB714
:1012E00026960FB6F894DEBF0FBECDBFDF91CF912B
:1012F0000895089508950C947A090C947B090E942E
:101300007D0960930F0270931002809311029093F5
:1013100012020C941B090C947F090F931F930091E8
:101320000F02109110022091110230911202602BD5
:10133000712B822B932B1F910F910C947F090F938C
:101340001F9300910F021091100220911102309111
:10135000120260237123822393231F910F910C9417
:101360007F090F931F9300910F021091100220919B
:1013700011023091120260277127822793271F9153
:101380000F910C947F090C9483030E94C30960930E
:101390000B0270930C0280930D0290930E020C943A
:1013A0001B0960E070E0CB010C94C5096115710563
:1013B0008105910529F481E0442361F080E00895DE
:1013C000DC01CB0104C0B695A795979587954A9502
:1013D000D2F7817008950F931F9341E050E060E0D1
:1013E00070E08A019B0104C0000F111F221F331FF0
:1013F0008A95D2F7C901B8011F910F910C94C509C4
:101400000F931F9341E050E060E070E004C0440F90
:10141000551F661F771F8A95D2F780910B02909116
:101420000C02A0910D02B0910E028A019B01082BC3
:10143000192B2A2B3B2BC901B8011F910F910C943A
:10144000C5090F931F9341E050E060E070E004C0D5
:10145000440F551F661F771F8A95D2F74095509508
:101460006095709580910B0290910C02A0910D02F5
:10147000B0910E028A019B01082319232A233B23E2
:10148000C901B8011F910F910C94C5090F931F93C7
:1014900041E050E060E070E004C0440F551F661F5B
:1014A000771F8A95D2F780910B0290910C02A09140
:1014B0000D02B0910E028A019B01082719272A27E5
:1014C0003B27C901B8011F910F910C94C5090F93D7
:1014D0001F9300910B0210910C0220910D0230918C
:1014E0000E02602B712B822B932B1F910F910C946A
:1014F000C5090F931F9300910B0210910C022091CC
:101500000D0230910E0260237123822393231F91D9
:101510000F910C94C5090F931F9300910B0210912A
:101520000C0220910D0230910E0260277127822754
:1015300093271F910F910C94C50908952DE0929F58
:10154000800D1124E82FE695E695E695877051E029
:1015500001C0550F8A95EAF785E0E89FF001112454
:10156000E252FE4F20E030E070E04081CB01022EDD
:1015700002C0969587950A94E2F781708195842739
:101580008523842781932F5F3F4F2530310569F7ED
:1015900008952DE0929F800D1124682F6695669521
:1015A0006695982F977085E0689FB001112440E000
:1015B00050E080E0FB01E40FF51FE252FE4F208176
:1015C00030E0092E02C0369527950A94E2F7217083
:1015D0003327042E01C0220F0A94EAF7822B4F5FB3
:1015E0005F4F4530510531F70895BF92CF92DF929A
:1015F000EF92FF920F931F93CF93DF938C01C090D4
:101600000B02D0900C02E0900D02F0900E0280913F
:101610000F0290911002A0911102B0911202C82AFB
:10162000D92AEA2AFB2ACFE1D0E0D701C6010C2E45
:1016300004C0B695A795979587950A94D2F780FD33
:1016400004C0219790F7B12C07C0BC2EB8018C2F95
:101650000E9411130197A9F38B2DDF91CF911F9158
:101660000F91FF90EF90DF90CF90BF900895CF93B0
:10167000DF93EC010E94F50ABE010E941113DF9175
:10168000CF9108951F93CF93DF93EB019091DD01EC
:10169000992321F0CB010E94370B13C0882349F016
:1016A000CB010E94F50A182F682FCE010E949E0AD6
:1016B00004C0CB010E94C90A182FBE01812F0E94CD
:1016C0001113DF91CF911F9108951F93CF93DF9353
:1016D000C091130216E080911402C81799F0D0E06F
:1016E0001C9FF0011D9FF00D1124EB5EFD4F40810A
:1016F000518162817381848195810E94690921965B
:10170000C770E9CFDF91CF911F91089540914502B5
:1017100050914602609147027091480280914902BF
:1017200090914A020C94690920911302909114023D
:1017300056E02917A9F030E0529FF001539FF00DB9
:101740001124EB5EFD4F7181761306C07081781312
:1017500003C07281741306C02F5F3F4F2770E9CF1B
:1017600080E0089581E00895DF92EF92FF920F9359
:101770001F93CF93DF9380914A0282958F7009F077
:1017800063C080914702882309F45EC0C0911302B0
:1017900086E0D82E80911402C81709F455C09091A4
:1017A000450240914602209148023091490221159C
:1017B000310531F04F3F31F481E09F3F19F403C010
:1017C00081E001C080E0D0E080FD3BC0DC9E800174
:1017D000DD9E100D1124F801EB5EFD4F8181841315
:1017E00030C0808189132DC0828181112AC0E3809D
:1017F000F480E21AF30A60E085E492E00E94470474
:1018000065E472E00E945A03E816F906D0F480916C
:101810004A028F70806180934A02F801E65EFD4FB4
:1018200080818F708061808385E492E00E94D90876
:10183000DF91CF911F910F91FF90EF90DF900C946B
:10184000650B2196C770A6CFDF91CF911F910F91A5
:10185000FF90EF90DF9008954F925F926F927F928A
:101860008F929F92AF92BF92CF92DF92EF92FF92B0
:101870000F931F93CF93DF93CDB7DEB761970FB66A
:10188000F894DEBF0FBECDBF8C0185E0F801DE010C
:101890001D9601900D928A95E1F7D8014C90119612
:1018A0005C90119712966C9012971396ED90FC90A5
:1018B000149760E085E492E00E9447044C01909107
:1018C000450280914602209148023091490221153B
:1018D000310531F08F3F31F481E09F3F19F403C0AF
:1018E00081E001C080E080FDE7C185E4C82E82E090
:1018F000D82E709047025701A21AB30A60E07720F1
:1019000009F465C1C6010E944704B6010E945A034A
:1019100020914A02207FA816B90608F00EC19091C6
:1019200045023091460240914802509149022111EE
:10193000A5C0452B31F03F3F31F481E09F3F19F4C2
:1019400003C081E001C080E080FD1CC0F8018181FE
:10195000831318C08081891315C0762C611012C0C2
:1019600080914A028F70806180934A020E94860BA8
:1019700085E492E00E94D90880914A02D801159628
:101980008C93B4C165E472E0C4010E945A03843FA1
:10199000914030F1E114F10439F0EFEF5E1206C02E
:1019A00081E04E1203C003C081E001C080E080FDF1
:1019B00003C081E0862502C080E090E080FF10C077
:1019C000462D652D842D0E94940B882349F085E4D3
:1019D00092E00E94D908E5E4F2E086E0DF01BDC0B4
:1019E000EF2839F0BFEF5B1206C081E04B1203C055
:1019F00003C081E001C080E080FD03C081E0862556
:101A000002C080E090E0E82FE170FE2E80FF2CC045
:101A1000462D652D842D0E94940B782E811124C0B3
:101A20004D865E868D859E850E94370B292F2295D7
:101A30002F70223018F0243090F405C09F7059F0B8
:101A4000811109C053C19F7031F0D80115969C9146
:101A5000907F09F44BC1805E883008F447C1C8010B
:101A60000E94D9087F2C42C1762C662009F43EC121
:101A700080914A02816080934A0274C0452B31F004
:101A80003F3F31F481E09F3F19F403C081E001C082
:101A900080E080FD0CC0F8018181831308C0808143
:101AA000891305C0611003C080914A02D3C0C801E8
:101AB0000E9452098823D9F16620C9F120914A0277
:101AC000822F82958F7090E0029774F0809145028A
:101AD0009091460298878F831986FB86EA862C8729
:101AE000CE0107960E94D90886E0F801A5E4B2E08D
:101AF00001900D928A95E1F70E94B40B0E94860B2B
:101B000019C090914502209146024091480250919F
:101B10004902452B49F12F3F49F581E09F3F31F5BF
:101B200080FF26C0C8010E945209811138C0C80137
:101B30000E94D90877247394D9C02111E2CF7E2D59
:101B4000F98AE88AA201662D89890E945A0985E4EA
:101B500092E00E94D90886E0D6011D928A95E9F7A5
:101B60000E94860B712CC2C081E0DACF80E0D8CF12
:101B7000F80181818213D6CF80818913D3CF611080
:101B8000D1CF80914A028583C8010E94D90886E09E
:101B9000E5E4F2E0DF011D928A95E9F7A7C066202F
:101BA00031F220914A02822F82958F7090E0029745
:101BB0000CF49ACF80914502909146029A838983D2
:101BC0001B82FD82EC822E83CE0101968BCF85E4B1
:101BD00092E00E94470465E472E00E945A03A8164E
:101BE000B90608F05BC0762C662009F4A0CF90916E
:101BF0004502209146024091480250914902452BEE
:101C000031F02F3F31F481E09F3F19F403C081E0B0
:101C100001C080E080FD34C0F8018181821330C0B2
:101C2000808189132DC020914A0220FD20C0822F7F
:101C300082958F70482F50E041155105C1F02583E2
:101C40004F30510541F08F5F982F9295907F822FF2
:101C50008F70892B8583C8010E94D90886E0F8011E
:101C6000A5E4B2E001900D928A95E1F73DC086E0CF
:101C7000F801A5E4B2E001900D928A95E1F736C033
:101C8000C8010E94520981112FCF80914A028160C0
:101C900080934A02C8010E94D90828C07E2DF98A83
:101CA000E88AA201662D89890E945A0986E0D60138
:101CB0001D928A95E9F718C0662009F438CFC8014B
:101CC0000E945209782E882309F431CF86E0F8016A
:101CD000A5E4B2E001900D928A95E1F785E492E0E7
:101CE0000E944A050E94B40B0E94860B872D6196C4
:101CF0000FB6F894DEBF0FBECDBFDF91CF911F911D
:101D00000F91FF90EF90DF90CF90BF90AF909F909A
:101D10008F907F906F905F904F9008951F93CF9317
:101D2000DF93CDB7DEB72C970FB6F894DEBF0FBEAA
:101D3000CDBF4F83588769877A878B879C87CE0171
:101D400007960E942C0C8823D1F09F8188852A85D4
:101D50003B85232B31F08F3F31F481E09F3F19F415
:101D600003C081E001C080E080FD47C04F815885FD
:101D700069857A858B859C850E9469093EC086E0CD
:101D8000FE013796DE01119601900D928A95E1F7DA
:101D9000FF81E8856A857B856115710531F0EF3F2C
:101DA00031F481E0FF3F19F403C081E001C080E01D
:101DB00080FD23C02091140230E0C9010196877094
:101DC00099274091130250E084179507F1F1F983A8
:101DD000EA837D836C8396E0929FD001939FB00D40
:101DE0001124AB5EBD4FFE01319601900D929A9584
:101DF000E1F7809314020E94650B16E080911302B4
:101E000090911402891771F1189FC00111248B5E03
:101E10009D4F0E942C0C882329F1E09113021E9FF4
:101E2000F0011124EB5EFD4F40815181628173818D
:101E3000848195810E9469098091130290E0019646
:101E40008770992780931302D9CF0E94330910928B
:101E5000140210921302E5E4F2E086E0DF011D9225
:101E60008A95E9F72C960FB6F894DEBF0FBECDBF6A
:101E7000DF91CF911F9108958091530285958595AB
:101E8000859508958091530287700895909153022B
:101E9000977081E009F480E0089580915E020895D2
:101EA00090915E02892B80935E02089580959091B7
:101EB0005E02892380935E02089510925E02089567
:101EC00080915D02089590915D02892B80935D025F
:101ED0000895809590915D02892380935D02089515
:101EE00010925D02089580915402089508950C9413
:101EF000760F0C94770F9091AE0292FD08C09091EE
:101F00005402981721F0809354020C94790F08958D
:101F100080915402882329F01092540280E00C949E
:101F2000790F0895CF93DF93E0913001F091310163
:101F300080915E028083E0913001F09131019081C7
:101F400080915D02892B808380915402882381F0E7
:101F5000E0913001F09131019081892B8083809153
:101F60003001909131010E941A2181110E94880F45
:101F7000C0913001D091310148E050E06BE472E053
:101F8000CE010E947B29892B69F088E0FE01ABE439
:101F9000B2E001900D928A95E1F7CE01DF91CF91E9
:101FA0000C94D520DF91CF9108950C94760F9091E9
:101FB000AE0292FD10C098E0899F90011124262B5B
:101FC000209353020E94000A8091530285958595C3
:101FD00085950C94D50F0C94000A1092530280E062
:101FE0000C94D50F20915302809582238093530245
:101FF000982F977099F430E0482F082E000C550B5D
:102000002417350759F09091AE0292FD07C08595CF
:10201000859585950E94210A0C94ED0F0895909165
:10202000AE0292FB222720F9281769F080FB92F973
:102030009093AE028091AD029091AE020E945D102D
:1020400082E00C94F20F08958091AE0282FB882703
:1020500080F991E089270C940F1081E00C940F1007
:1020600080E00C940F106FEF7FEF80E090E00C9415
:10207000BA2980E090E00E94962921E0893E9E4F97
:1020800009F020E0822F089582E090E00C948829E6
:1020900083E090E00C948829CF9384E090E00E9444
:1020A0008829C82F82E290E00E9488292C2F30E0F6
:1020B000A901582BCA01CF910895CF93C92F682F3A
:1020C00084E090E00E949C296C2F82E290E0CF9106
:1020D0000C949C29AB01BC018FE090E00C94AE29DC
:1020E000AB01BC0183E190E00C94AE2960E070E0AC
:1020F000CB010C94701060E070E0CB010E946A107C
:102100000C94761069EE7EEF80E090E00E94BA2990
:1021100060E082E090E00E949C2960E083E090E033
:102120000E949C2910920F0210921002109211022C
:102130001092120260E084E090E00E949C2960E02E
:1021400082E290E00E949C2960E085E090E00E949D
:102150009C2960E086E090E00E949C296FEF87E078
:1021600090E00E949C2940E050E0BA0188E090E0B5
:102170000E94AE2960E08DE090E00E949C2940E042
:1021800050E0BA0188E190E00E94AE2960E087E16A
:1021900090E00E949C2940E050E0BA018CE190E080
:1021A0000E94AE2960E070E080E290E00E94BA29CF
:1021B00040E050E0BA0188E190E00E94AE290C9422
:1021C0007B100C948210682F8EE090E00C949C2978
:1021D0000E940F22609371027093720280937302C7
:1021E0009093740260936D0270936E0280936F02FD
:1021F0009093700208950E940F2260937102709371
:1022000072028093730290937402609369027093D8
:102210006A0280936B0290936C02089585B7806880
:1022200085BF85B7806885BF089581E008950C94C7
:10223000151108950C9419110C946E030C94191136
:102240000C941E110C9419110E940E118DEE93E145
:102250000E94BF200E9422110C9420110E941A118A
:102260000C9419110E9407140C94E4040E94FA21A2
:102270000E94EC140E9432110E94FD1A0E948B1DD4
:102280000C941C115F926F927F928F929F92AF92EB
:10229000BF92CF92DF92EF92FF920F931F93CF9353
:1022A000DF93CDB7DEB72A970FB6F894DEBF0FBE27
:1022B000CDBF0E940115C82E81110E94E8103FE594
:1022C000832E32E0932E00E010E0502E802F0E94EB
:1022D0002B145C01F401619071904F0168267926FE
:1022E00061147104B1F40F5F1F4F0530110569F7D8
:1022F0008FEF89838A831B820E9403228160782F5B
:102300009D838C8349815A816B818D810E94000558
:102310003AC08091750281FD0E943414D12CEE24C4
:10232000E394F12CC3018E219F21892B29F10E9476
:1023300017118823A9F0DE825F82AE20BF2081E0E2
:10234000AB2809F480E088870E9403228160782FFF
:102350009A8789874E815F8168858A850E940005FA
:10236000000F111FF801E15AFD4F80819181E8268D
:10237000F926F182E08207C0D394EE0CFF1CFDE049
:10238000DF12D0CFB0CF81E0C11001C080E02A962B
:102390000FB6F894DEBF0FBECDBFDF91CF911F9176
:1023A0000F91FF90EF90DF90CF90BF90AF909F90F4
:1023B0008F907F906F905F9008950E9442110E94CD
:1023C00041200E94301B0E949E1D81110E94FB1023
:1023D0000E9408170C94F504CF93DF930E94161304
:1023E000EC01811521E5920708F045C0811530E523
:1023F000930708F094C0883E910528F5803E91052A
:1024000008F0F8C0883A910570F4853A910508F013
:102410007CC08130910509F475C008F4E8C00497C8
:1024200008F0E8C0E4C08F3B910508F0E0C0C85A4E
:10243000D0E0CC0FDD1FC058DE4F0990D881C02DF1
:10244000CE019464D8C0811540E2940758F48115F8
:1024500051E0950708F0CEC08D3E910508F4C7C045
:102460009065C9C0C11580E4D80708F4C0C0DF700A
:10247000CE01906AC0C0811525E59207A8F48115A8
:1024800034E5930708F095C0811543E5940708F0FB
:102490007BC0811552E5950708F061C0D82FCC2785
:1024A000CE01816F906AA7C0C11589E5D807A0F455
:1024B000C11528E5D20708F082C0C11536E5D3075B
:1024C00008F095C08C2F0E94AA138F7190E0D82F2E
:1024D000CC27CE0190628FC0C1154AE5D40708F41D
:1024E00074C0CE0190568115904208F080C08D2FA7
:1024F0008F710E94AA13DD27D0628F71AE01582B15
:10250000CA0179C081E090E076C0C55AD0E0C255DA
:10251000DE4F8881C82FD0E0CE0190646CC074E09B
:10252000969587957A95E1F7282F23703C2F337085
:1025300081E090E002C0880F991F3A95E2F79C680D
:10254000AC01522B9A019C2F9F709695969550E264
:10255000959FE0011124C9018C2B9D2B4CC08370E9
:10256000992721E030E002C0220F331F8A95E2F75D
:102570009C2F9695969580E2989FE0011124C22B9E
:10258000D32BCE019C6837C08370992721E030E0BF
:1025900002C0220F331F8A95E2F79C2F96959695DD
:1025A00040E2949FE0011124C22BD32BCE019A6804
:1025B00022C0D82FCC27CE01846F906A1CC0DC2F9C
:1025C000CC27CE01806F906A16C08C2F8F700E942E
:1025D000AA1394E0D695C7959A95E1F7CF70D0E00D
:1025E000DC2FCC27D0699E01282BC90104C080E0D4
:1025F00090E001C0CE01DF91CF91089521E4829F48
:10260000C0011124FC012DE0729FE00DF11D112489
:10261000E60FF11DEE0FFF1FE852FF4F85919491D9
:1026200008950E94FE120E94EC11089582389105CF
:1026300069F1B0F48133910509F46DC048F4893231
:10264000910509F463C08A32910509F469C00895BF
:102650008533910509F455C089339105B9F0089582
:10266000833E910569F138F4803E9105B1F0823ED8
:10267000910509F10895863E9105A9F1873E9105DE
:10268000B9F1843E910509F064C023C02091AD02E8
:1026900020FD4FC021FD4DC008958091AD0280FD09
:1026A00044C08091AE0280FF44C08091AD0284FDA1
:1026B00042C083EE4DC08091AD0282FF38C0F5CF9D
:1026C0008091AD0282FD33C08091AE0280FD31C0A9
:1026D000ECCF8091AE0281FF32C08091AD0284FDCB
:1026E0002AC087EE35C08091AD0283FF26C0F5CFAA
:1026F0008091AD0283FD21C08091AE0281FD1FC09B
:10270000ECCF8091AD0285FD1CC01DC08091AD0253
:1027100085FD19C016C08091AD0286FD16C017C098
:102720008091AD0286FD13C010C089E311C082EE16
:102730000FC080EE0DC080E00BC086EE09C084EEB5
:1027400007C089E205C085E303C08AE201C081E3D6
:1027500090E008959091AD0292FF0DC0282F28714E
:10276000283019F4877F846006C0282F2471243014
:1027700011F48B7F886093FF0DC0282F28712831BA
:1027800019F4877E846106C0282F2471243111F446
:102790008B7E88612091AE0220FF0DC0382F3871EA
:1027A000383019F4877F816006C0382F317131309D
:1027B00011F48E7F886021FF0DC0282F28712831E9
:1027C00019F4877E816106C0282F2171213111F40F
:1027D0008E7E886194FD877E089580E008950C9434
:1027E00033100E9401158FE39CE90197F1F700C0B7
:1027F00000000E94011580E00E942B1480FF04C09D
:102800000E94EF130C94502208950C94F1130E942F
:102810003910811102C00E94E1100E94441080937F
:1028200075020E944C109093AE028093AD020E94FC
:1028300005140E944810682F70E080E090E00E942C
:102840008B0960910B0270910C0280910D029091A6
:102850000E020C94C309E82FF0E0EE0FFF1FE754BF
:10286000FD4F808191810895089580EA8A95F1F75E
:10287000089500C008950C94351408950C943D14E7
:102880000C943E140C943D140C944214F894E82FCC
:10289000E295EF70F0E031A1282F2F7081E090E0F9
:1028A00001C0880F2A95EAF7982F9095932391A35A
:1028B00092A1892B82A3789408950F931F93CF93AD
:1028C000DF93CEEBD1E089918F3F11F00E94461447
:1028D00081E0C33CD807B9F7C1EBD1E00EEB11E0C2
:1028E00089918F3F11F00E9446140C171D07C1F704
:1028F000DF91CF911F910F910895BF92CF92DF92F8
:10290000EF92FF920F931F93CF93DF938C01C62F0B
:10291000D0E0CE0182549E4F6C01FC0190819F3F1C
:1029200009F450C0B62EF894E92FE295EF70F0E06C
:1029300081A19F7021E030E001C0220F9A95EAF753
:10294000822B81A382A12095282322A378940E9420
:102950003914E1EBF1E04EEB51E021E030E0E12C05
:10296000F12C61916F3F89F0A62FA295AF70B0E076
:1029700090968C9190E06F7002C0959587956A95BE
:10298000E2F780FD02C0C90102C080E090E0E82AC1
:10299000F92A220F331F4E175F0719F7F6018081BE
:1029A0008F3F11F00E94461461E0E114F10409F434
:1029B00060E08B2D0E943B14CC0FDD1FC00FD11F98
:1029C000F982E882DF91CF911F910F91FF90EF90F4
:1029D000DF90CF90BF9008950E945D148AE0E9EBEC
:1029E000F2E0DF01982F1D929A95E9F7EFEAF2E005
:1029F000DF011D928A95E9F785E00E944C150C9441
:102A00005D04FF920F931F93CF93DF93CDB7DEB793
:102A10002A970FB6F894DEBF0FBECDBF8E010F5FB1
:102A20001F4F8AE0F80111928A95E9F7F12C6F2D7A
:102A3000C8010E947D14F394F5E0FF12F8CF4AE03C
:102A400050E0B8018FEA92E00E947B29FF24F394C2
:102A5000009709F4F12C892B41F08AE0F801AFEAE4
:102A6000B2E001900D928A95E1F72F2D45E069EBD8
:102A700072E08FEA92E00E944D150E945F048F2D54
:102A80002A960FB6F894DEBF0FBECDBFDF91CF916F
:102A90001F910F91FF9008950895FF920F931F9338
:102AA000CF93DF93F82E092F162FD72FC42F222371
:102AB00049F081E0809378020E940322909377028C
:102AC00080937602809178028823D9F080917602F3
:102AD000909177020E941B22059798F0EF2DF02F1E
:102AE000A12FBD2F80E090E04C2F50E08417950778
:102AF00034F4219131912D933D930196F7CF1092AB
:102B00007802DF91CF911F910F91FF9008950E945D
:102B100006240E9436110C9412240E9416240E944E
:102B2000DD110C9430240E94A1210E94ED230E940B
:102B300024110E9487150E948D150E942E11FBCF33
:102B400080917F0280FF06C06091370170E0660FC0
:102B5000771F26C081FF04C06091370184E005C063
:102B600082FF07C06091370188E0689FB00111249F
:102B700017C090917E029923D1F06091360196178B
:102B800088F72091370188E0289F90011124929FB7
:102B9000A001939F500D112470E0CA010E94542996
:102BA0006038710540F46115710519F406C068E0DC
:102BB00070E0862F08958FE7089581E00895809151
:102BC0007F0280FF08C06091330170E075956795C2
:102BD0007595679521C081FF06C06091330170E053
:102BE0007595679519C082FF04C06091330170E04C
:102BF00010C090917D02992399F06091320196174F
:102C0000A0F780913301899FC001112470E00E94D8
:102C100054296038710540F46115710519F406C036
:102C200061E070E0862F08958FE7089581E00895B0
:102C30008D3E21F40E94A015819504C08E3E29F49A
:102C40000E94A0158093830208958F3E21F40E9474
:102C5000A015819504C0803F29F40E94A01580939F
:102C600082020895893F19F40E94DF1505C08A3F4A
:102C700031F40E94DF1581958093840208958B3F83
:102C800021F40E94DF15819504C08C3F29F40E9435
:102C9000DF158093850208959FE0980F983078F4AF
:102CA00021E030E0A90102C0440F551F9A95E2F7D8
:102CB000CA0190918102892B8093810208958D3FF2
:102CC00021F480917F0281600BC08E3F21F48091BE
:102CD0007F02826005C08F3F29F480917F0284606B
:102CE00080937F0208958D3E39F49091830297FF7F
:102CF00035C01092830259C08E3E29F49091830210
:102D00001916BCF32BC0909182028F3E29F497FFD5
:102D100025C01092820249C0803F19F41916CCF3E5
:102D20001DC090918402893F29F41916BCF41092B9
:102D300084023BC08A3F19F497FF10C0F8CF8B3F45
:102D400039F49091850297FF09C0109285022DC039
:102D50008C3F21F4909185021916BCF39FE0980FE7
:102D6000983080F421E030E0A90102C0440F551FE3
:102D70009A95E2F7CA018095909181028923809308
:102D8000810213C08D3F21F480917F028E7F0BC0A2
:102D90008E3F21F480917F028D7F05C08F3F29F403
:102DA00080917F028B7F80937F02809182028111CC
:102DB00006C080918302811102C010927E02809130
:102DC0008402811106C080918502811102C0109297
:102DD0007D0208950E94032220918202211104C0E5
:102DE00020918302222321F090937C0280937B0226
:102DF00020918402211104C020918502222321F018
:102E000090937A028093790280E892E00C94E0201B
:102E1000EF92FF920F931F93CF93DF9300D000D0D8
:102E200000D0CDB7DEB786E0E0E8F2E0DE01119633
:102E300001900D928A95E1F7E0908202F090830272
:102E400000918402109185021092820210928302F6
:102E50001092840210928502E11003C0FF2009F451
:102E60005DC080917B0290917C020E941B22AC018C
:102E700090917E02992339F02091380130E0241797
:102E8000350758F04BC0209139018AE0289F900106
:102E900011242417350718F041C09F3F19F09F5F98
:102EA00090937E02EE2061F00E94A0151E1414F093
:102EB0009FEF01C091E0989F902D11249093820282
:102EC000FF2061F00E94A0151F1414F09FEF01C0B5
:102ED00091E0989F902D112490938302309182026B
:102EE0003323E1F0209183022223C1F045EB340328
:102EF000C0011124992319F09093820203C081E04C
:102F00008093820235EB2303C0011124992319F029
:102F10009093830203C081E080938302011103C078
:102F2000112309F45DC08091790290917A020E9488
:102F30001B22AC0190917D02992339F0209134013C
:102F400030E02417350758F04BC0209135018AE056
:102F5000289F900111242417350718F041C09F3F86
:102F600019F09F5F90937D02002361F00E94DF15AE
:102F7000101614F09FEF01C091E0989F902D11243E
:102F800090938402112361F00E94DF15111614F052
:102F90009FEF01C091E0989F902D1124909385029E
:102FA000309184023323E1F0209185022223C1F085
:102FB00045EB3403C0011124992319F09093840246
:102FC00003C081E08093840235EB2303C001112408
:102FD000992319F09093850203C081E080938502C4
:102FE0008091820281110BC080918302811107C000
:102FF00080918402811103C08091850281110E9419
:10300000EA16EB82FC820D831E8386E0FE01319678
:10301000A0E8B2E001900D928A95E1F726960FB6EE
:10302000F894DEBF0FBECDBFDF91CF911F910F91FE
:10303000FF90EF900895E0E8F2E086E0DF011D9256
:103040008A95E9F710927E0210927D0210927F021B
:103050000895EF92FF920F931F93CF93DF938B010D
:10306000682F11110AC0442329F0E82FF0E0EC5139
:10307000FC4F6491762F862F75C0212F30E0E82F0A
:10308000F0E0442321F0EC51FC4FE491F0E046E005
:10309000049FC0011124CFEFD0E0BE010E9440295F
:1030A0004BEA4603C001479F900D1124800F911DEC
:1030B000800F911D982F990F890FAE01421B530B62
:1030C0004E9FD0014F9FB00D5E9FB00D11249B2FDE
:1030D000189FA0011124452F55278E01041B150BA5
:1030E0000E9FA0010F9F500D1E9F500D11247E01B9
:1030F000E81AF108E29E8001E39E100DF29E100D89
:103100001124212F3327C21BD30BCE9F9001CF9FB9
:10311000300DDE9F300D112462307105A9F048F4A6
:103120006115710569F061307105C9F48B2F752F38
:103130000DC06430710581F058F06630710579F486
:103140007E2F8B2F932F0DC0832F7B2F9E2F09C097
:103150008E2F7B2F952F05C08E2F732F02C07E2FB1
:10316000852F692FDF91CF911F910F91FF90EF90E5
:10317000089541E00E94291808950895823070F45E
:10318000262F30E0280F311D233031053CF4809389
:103190003C01860F80933D0160933E0108950E949B
:1031A000B9180895CF93DF93762FE901682F842F04
:1031B0000E94CF18798368838A83DF91CF91089525
:1031C000F90181836083428308958091C302282F8F
:1031D000269530E02115310519F48170826005C013
:1031E0002630310524F081708A608093C3020895EF
:1031F00088E090E00C949029CF92DF92EF92FF92BA
:103200006B017C010E94E518B701A60188E090E0FF
:10321000FF90EF90DF90CF900C94AE29E3ECF2E0BA
:1032200083E0808311828FEF8283838314826081A5
:103230007181828193810C94FC188091C30280FF7C
:1032400002C08695089580E008959091C70293305A
:1032500018F49F5F9093C702882351F06091C302D6
:103260007091C4028091C5029091C6020C94FC1822
:10327000089581E00C9425199091C702992319F0C3
:1032800091509093C702882351F06091C3027091CE
:10329000C4028091C5029091C6020C94FC18089556
:1032A00081E00C943C1970E00C940F1C60913B0180
:1032B0008091C30280FF0AC080913A0123E0829F7F
:1032C000C001112488539D4F0C94531980913C01E7
:1032D00090913D01891780F7E82FF0E09F01220FC0
:1032E000331FE20FF31FE853FD4F11821082128249
:1032F0008F5FF0CF9091C30290FF16C090913C0178
:1033000020913D01921770F4E92FF0E0DF01AA0F40
:10331000BB1FEA0FFB1FE853FD4F8183608342838D
:103320009F5FF0CF0C9456190895CF93DF9300D090
:103330001F92CDB7DEB79091C30290FF0AC09E01E5
:103340002F5F3F4F0E94D2184B8169818A810E9472
:103350007A190F900F900F90DF91CF910895CF932E
:10336000DF93EC01EC81F0E0EC51FD4F4491E3EC94
:10337000F2E0628181810E9495198C818F5F8C833C
:10338000DF91CF910895EF92FF920F931F93CF9308
:10339000DF9300D01F92CDB7DEB7F82E062F142F83
:1033A000E22E8091C30280FF2DC0E82FE695F0E069
:1033B000ED53FE4F908190938D028E7F823061F4A9
:1033C0009E012F5F3F4F8F2D0E94D2184B81698144
:1033D0008A810E947A1904C0923011F41091C602B9
:1033E000F092C4020093C5021093C602EE2051F081
:1033F0006091C3027091C4028091C5029091C6028F
:103400000E94FC180F900F900F90DF91CF911F91A9
:103410000F91FF90EF900895E3ECF2E09181282F57
:103420004381628188E0890F0C94C31981E00C9478
:103430000C1AE3ECF2E09181282F4381628188EF3E
:10344000890F0C94C31981E00C94191AE3ECF2E093
:10345000628121E1620F08F46FEF282F438181819F
:103460000C94C31981E00C94261AE3ECF2E062811B
:1034700021E1621B08F460E0282F438181810C94D4
:10348000C31981E00C94351AE3ECF2E0438121E1A9
:10349000420F08F44FEF282F628181810C94C319E9
:1034A00081E00C94441AE3ECF2E0438121E1421BF9
:1034B00008F440E0282F628181810C94C31981E0D7
:1034C0000C94531A20E00C94C319E3ECF2E08081D1
:1034D0008E7F808360817181828193810E94FC183C
:1034E00010928E022FEF80E792E0215080409040B2
:1034F000E1F700C000000C9456196091C302669574
:1035000070E041E050E08FE391E00E946E29892B4A
:1035100019F481E080938E020E9403229093870227
:103520008093860208959091C30290FF35C09170F8
:10353000811102C0926006C0863010F09A6002C00D
:10354000880F982B9093C302662351F06091C302B9
:103550007091C4028091C5029091C6020E94FC182D
:103560006091C302669570E041E050E08FE391E026
:103570000E946E29892B19F010928E0202C00E94BF
:103580007D1A81E0809389024091C6026091C50254
:103590008091C4020C94621A0895682F9091C3021E
:1035A000969581E0890F863008F081E00C94931A9B
:1035B00081E00C94CD1A682F9091C30296958FEFFD
:1035C000890F09F485E00C94931A81E00C94DB1ABE
:1035D00061E00C94931AE3ECF2E0808181608083D7
:1035E00086950C94E81A8091C30280FD0C94651AAC
:1035F0000C94EB1A60E00C94931A80918C02811168
:103600002EC00E943910811104C00E94E1100E9456
:103610000E190E94F8186093C3027093C40280933D
:10362000C5029093C6026E7F61F40E940E190E943B
:10363000F8186093C3027093C4028093C5029093FC
:10364000C6020E94E51810928E028091C30280FF8C
:1036500003C086950E94FA1A81E080938C02089537
:103660000F931F93CF93DF9380918E02882309F4E9
:1036700040C080918D02E091C302E695E81BE09383
:103680008802823049F4F0E0E052FD4FE491CE2F01
:10369000D0E00FEA19E104C0C0EDD7E00DEB18E16E
:1036A00080918902882361F0109289020E9403228E
:1036B000909387028093860210928B0210928A0266
:1036C0000E940322E0918602F09187028E1B9F0BDD
:1036D0008F3F9F4770F4CE0FDF1FD0938702C093B8
:1036E000860286E892E0F801DF91CF911F910F9159
:1036F0000994DF91CF911F910F910895882311F0C4
:10370000FA0101C0FB0109940E941D19823030F0BA
:103710000E941D19853010F40C94D81A82E00C9484
:10372000E81A1F93CF93DF93FB011281111172C02E
:10373000EC010E944D0F8272CA3CFCE5DF0709F4E0
:1037400057C0C8F4C63CECE5DE0709F442C048F4B3
:10375000C43C9CE5D90789F1A8F5C33CDC4551F18F
:1037600027C0C83C9CE5D907C9F1E8F546E15AE114
:1037700063E27AE12BC0CE3CFCE5DF0709F447C0E9
:1037800050F4CC3CECE5DE07C1F1E0F540E55AE150
:103790006FE57AE11BC0C73D8CE5D80730F4C03D2A
:1037A000DC45C0F50E94841B35C0CE35DD4591F166
:1037B00011E030C00E94F31A2DC045EE5AE168EDC9
:1037C0007AE104C048ED5AE165EE7AE10E947E1B81
:1037D00021C043E25AE166E17AE1F8CF41E45AE1DF
:1037E00062E37AE1F3CF42E35AE161E47AE1EECFBA
:1037F0004FE55AE160E57AE1E9CF40E559E169E357
:1038000079E1E4CF49E359E160E579E1DFCF81E097
:103810000E94E81A812FDF91CF911F910895279A76
:1038200025B12F7735B130684FB7F894FC01CB0143
:10383000880F991F680F791F6E0F7F1FE617F70714
:1038400089F0819198E035B9000000C087FF25B963
:10385000880F000000C000C000C025B900C09A95C4
:1038600091F7ECCF4FBF8FE594E00197F1F700C0DF
:1038700000000895CF93DF93EC01FB018281882340
:1038800009F43CC1C430FDE5DF0760F4CB3F9CE5A3
:10389000D90788F49E0122503C452431310508F0B7
:1038A0002EC109C0C236EDE5DE0729F0C63AFDE5B6
:1038B000DF0709F024C10E944C109093AE02809360
:1038C000AD02C1318CE5D80709F4C6C008F042C08A
:1038D000C930ECE5DE0709F49BC000F5C5308CE586
:1038E000D80709F485C078F4C330ECE5DE0709F4A5
:1038F00078C008F07AC0C230DC4509F0F5C080918C
:10390000AD028160EFC0C7309CE5D90709F478C0EB
:1039100008F07AC08091AD028061E4C0CD30FCE552
:10392000DF0709F487C058F4CB309CE5D90709F4C8
:1039300079C008F07BC08091AD0288606FC0CF3045
:10394000FCE5DF0709F480C008F082C08091AD0279
:10395000877FC8C0CE3F9CE5D90709F471C000F548
:10396000C531FCE5DF0709F485C068F4C3319CE587
:10397000D90709F475C008F095C00E9433098091F9
:10398000AD028F77AFC0CC3FFCE5DF07A9F108F0AF
:1039900054C0CB3FDC4509F0A7C08091AE0240C0C7
:1039A000C230EDE5DE0709F489C058F4C1158DE594
:1039B000D80709F45AC008F069C08091AE0282604D
:1039C0002FC0C236EDE5DE0709F47CC0C63AFDE53E
:1039D000DF0709F481C0C330DD4509F085C080E010
:1039E0006EC08091AD0282607DC08091AD0216C034
:1039F0008091AD02886076C08091AE0282604FC037
:103A00008091AD0280626EC08091AD0280646AC018
:103A10000E9433098091AD02806864C0846062C0F6
:103A200081603DC08091AD028E7F5CC08091AD020F
:103A30008D7F58C08091AD0216C08091AE0218C033
:103A40008091AE028D7F2BC08091AD028F7E4AC0E7
:103A50008091AD028F7D46C08091AD028F7B42C0C8
:103A60008091AD02877F8B7F3DC08091AE028D7FBC
:103A70008E7F15C08091AD0282FB222720F991E054
:103A8000922790FB82F990FB83F92CC08091AE02C3
:103A9000982F909591708E7F892B90FB81F9809360
:103AA000AE0222C00E9433098091AD0287FB22271B
:103AB00020F991E0922790FB87F914C081E00E94E1
:103AC000E31012C08091AD0284FB222720F991E01F
:103AD000922790FB84F906C08091AD02982F9095B3
:103AE00090FB80F98093AD028091AD029091AE027F
:103AF0000E945D100E94330980E001C081E0DF91E7
:103B0000CF9108958FE891E00197F1F700C0000090
:103B100008950C94630322982A9A2198299A0E9466
:103B2000821D83B182FB882780F9199902C090E039
:103B300001C092E0892B809391020895E091910257
:103B4000EE0FEE0FE093910243B142FB882780F91C
:103B500090E043B141FB222720F930E041FF02C051
:103B600022E030E0822B932B8E2B809391028F707A
:103B7000E82FF0E0E753FE4F908180919002890F8B
:103B80008093900284305CF080918F028F5F8093ED
:103B90008F0260E080E00E94891D21E001C020E0EA
:103BA000809190028D3F54F480918F0281508093D8
:103BB0008F0261E080E00E94891D21E080919002E7
:103BC000082E000C990B64E070E00E945429809349
:103BD0009002822F0895CF93DF9386319C4541F563
:103BE000EB010E944D0F982F8A8120913001309176
:103BF0003101882379F09A7A81E009F480E080939A
:103C00009202911102C069E201C065E3C9010E94FC
:103C10005C210AC080919202811102C069E201C058
:103C200065E3C9010E945E210E94920F80E001C0FD
:103C300081E0DF91CF910895AF92BF92CF92DF9252
:103C4000EF92FF920F931F93CF93DF937C015B0161
:103C5000C42FD22FFC0182818823F9F04093950272
:103C60000E940322909394028093930280E28C0F2F
:103C7000883008F06EC0C77081E001C0880FCA9517
:103C8000EAF7DF91CF911F910F91FF90EF90DF90B6
:103C9000CF90BF90AF900C9482068091950248130C
:103CA00035C080919302909194020E941B226C0176
:103CB000B701C5010E945A03C816D90638F510E2AB
:103CC0001D0FCD17B9F080E28C0F883040F4C7701B
:103CD00081E001C0880FCA95EAF70E948906183072
:103CE00058F581E09D2F977001C0880F9A95EAF7EB
:103CF0000E948206802F0E947906183050F5D770F6
:103D000081E001C0880FDA95EAF70AC080E28C0FE3
:103D10008830F8F4C77081E001C0880FCA95EAF7CF
:103D2000DF91CF911F910F91FF90EF90DF90CF9097
:103D3000BF90AF900C948906802FDF91CF911F9197
:103D40000F91FF90EF90DF90CF90BF90AF900C94C9
:103D50007906DF91CF911F910F91FF90EF90DF9047
:103D6000CF90BF90AF9008950F939C01CB01243F5B
:103D70004CE5340731F188F4293DFCE53F07D9F0E3
:103D80002A3D4CE5340779F1283D3C45A9F506E28A
:103D900021EE41EE68ED7CE52BC0263FFCE53F07B8
:103DA000E1F0A8F0273F3C4539F507E225EE46EE65
:103DB00067EF7CE51DC007E225EE45EE69ED7CE589
:103DC00017C006E221EE40EE64EF7CE511C007E289
:103DD00025EE44EE65EF7CE50BC006E221EE42EEF7
:103DE00066EF7CE505C008E221E045EE6AED7CE582
:103DF0000E941C1E80E008C0FC018281882319F00B
:103E00001092950201C081E00F910895CF93DF9346
:103E1000EC0181E0898B8F810E94500F88850E9480
:103E2000630F0E94920FEA81FB81CE0106963097C4
:103E300029F06C897D89DF91CF910994DF91CF9131
:103E40000895CF93DF93FC012081223041F4FB01E0
:103E5000EC01828193810E94DF0381E08B87DF91F7
:103E6000CF910895FC018081813021F4FB01808194
:103E7000918105C0823029F4FB01828193810C94E9
:103E8000DF030895FC018081813021F4FB018081F2
:103E9000918105C0823029F4FB01828193810C94C9
:103EA000F5030895EF92FF920F931F93CF93DF9343
:103EB000FC012285211136C0EC01E380F480F7E596
:103EC000FF1A26E12E9DC0012F9D900D1124DC01CB
:103ED000A050BF4F1496ED91FC9115978A5F9E4FAD
:103EE000309729F054966D917C915597099586E10C
:103EF0008E9D80018F9D100D112400501F4FF801E1
:103F000087810E94560FF80180850E94690F0E94E8
:103F1000920F188219861B861E821D8210929702AC
:103F200010929602DF91CF911F910F91FF90EF9029
:103F30000895DF92EF92FF920F931F93CF93DF9339
:103F4000FB0122812223C1F12091400130914101E6
:103F50002F3F3F4F89F18C01C0E0D1E0E12CF12CE3
:103F6000DD24D39480914001909141018E159F05ED
:103F70001CF18E818823D9F089859A858017910755
:103F800039F480919602909197020817190779F0F9
:103F9000DF861C870B878989811103C0CE010E94AF
:103FA000061FCE0106960E94521F0E94700F4FEF0F
:103FB000E41AF40A6696D6CFDF91CF911F910F9144
:103FC000FF90EF90DF900895EF92FF920F931F9371
:103FD000CF93DF939C0137552F3F310511F008F047
:103FE00048C040914001509141014217530724F4C9
:103FF0003093410120934001FB017C01828196E1D5
:10400000929F8001939F100D1124E801C050DF4F53
:10401000888B92818E81992311F1FA86E9868F5FD0
:104020008E830E9403229E878D870E94730F8F8349
:104030000E944D0F88870E94600F9885892B888782
:10404000E881F981C8018A5F9E4F309719F06C8929
:104050007D890995F0929702E09296020AC0882322
:1040600041F08989882329F0C8018A5F9E4F0E9408
:10407000521F81E0DF91CF911F910F91FF90EF9040
:1040800008957F928F929F92AF92BF92CF92DF92CC
:10409000EF92FF920F931F93CF93DF9300D000D046
:1040A00000D0CDB7DEB780914001909141010196DB
:1040B00009F451C0B12C86E1A82E96E0792ECE01EC
:1040C00001966C01EB2CF12C809140019091410103
:1040D0008E159F050CF43FC0AE9CF001AF9CF00D17
:1040E0001124E050FF4F828893888114910459F481
:1040F000D601272D1D922A95E9F7B6018185928573
:104100000E945A034C01AE9C8001AF9C100D1124FB
:1041100000501F4FD80116968C9116978823C9F02E
:104120001D968D919C911E970E941B2288169906C0
:1041300080F4F8018189811103C0C8010E94061F23
:10414000AE9CC001AF9C900D11248A5F9E4F0E94CF
:10415000521FB394B7CF26960FB6F894DEBF0FBEAA
:10416000CDBFDF91CF911F910F91FF90EF90DF9026
:10417000CF90BF90AF909F908F907F900895909335
:10418000DB018093DA01089590939D0280939C0255
:104190000895E0919C02F0919D02309721F00190EA
:1041A000F081E02D099480E00895E0919C02F09167
:1041B0009D02309721F00280F381E02D099408954B
:1041C000E0919C02F0919D02309739F022E0DC01F1
:1041D0002C930480F581E02D0994089520919A0292
:1041E00030919B022817390771F090939B028093BE
:1041F0009A02E0919C02F0919D02309721F0068096
:10420000F781E02D09940895209198023091990248
:104210002817390771F09093990280939802E091E2
:104220009C02F0919D02309721F00084F185E02DF1
:1042300009940895FC01329697E080E0915029F0AE
:1042400021912223D9F38F5FF9CF0895662349F096
:10425000FC01329608962191621729F0E817F907B8
:10426000D1F780E0089581E008959C01FC01329629
:104270009FEF80E04191461789F09F3F19F441116B
:1042800001C0982F8F5F8630A9F79F3F39F0F90161
:10429000E90FF11D97FDFA956283089508959C0139
:1042A0002A5F3F4FFC014281461301C012820196F2
:1042B00082179307B9F708950C9435210C944F2178
:1042C000029626E0FC0111922A95E9F708950895D7
:1042D0000C94672183E080939E020C9468218111E5
:1042E00002C081E001C082E080939E020C946821AC
:1042F0000C946F2181E080939E020C9468210C94B1
:104300007A2108950C9481210C9482210C948121AE
:104310000C9481210C948121CF930E9488210E94CA
:1043200001150E948621C0E08C2F0E942B14892B3E
:1043300029F4CF5FC530C1F780E001C081E0CF91A3
:10434000089508951F920F920FB60F9211248F9324
:104350009F93AF93BF9380919F02811113C080916F
:10436000CE029091CF02A091D002B091D10241969D
:10437000A11DB11D8093CE029093CF02A093D002D5
:10438000B093D102BF91AF919F918F910F900FBECB
:104390000F901F9018958091D602843031F10E94C1
:1043A000D50410929F0220E488E190E00FB6F894C3
:1043B000A895809360000FBE2093600083B7817F33
:1043C000846083BF83B7816083BF7894889583B707
:1043D0008E7F83BF0FB6F894A895809160008861A6
:1043E00080936000109260000FBE08950E94330910
:1043F0000C94D90482E084BD93E095BD9AEF97BDFB
:1044000080936E0008952FB7F8948091CE0290911A
:10441000CF02A091D002B091D1022FBF08952FB743
:10442000F8946091CE027091CF028091D002909169
:10443000D1022FBF08959C014FB7F8948091CE020E
:104440009091CF02A091D002B091D1024FBF821BB8
:10445000930B089578941F920F920FB60F92112428
:104460008F939F93AF93BF938091CE029091CF0291
:10447000A091D002B091D1020196A11DB11D8093EF
:10448000CE029093CF02A093D002B093D102BF91FD
:10449000AF919F918F910F900FBE0F901F90189525
:1044A00081E08093E00080E28093D8001092C90000
:1044B0008FE19EE40197F1F700C0000087E090EBE8
:1044C000DC018093DF029093E002A093E102B093BD
:1044D000E2029CE088E10FB6F894A8958093600012
:1044E0000FBE90936000FFCF8091AB0208950895B6
:1044F00022E02093E9002FEF3091E800215035FDB4
:1045000006C035ED3A95F1F700002111F5CF209165
:10451000E80025FF0BC040E050E066E070E00E943C
:10452000A2248091E8008E778093E8000895CF93CD
:10453000DF9321E02093E9002FEF3091E800215034
:1045400035FD06C035ED3A95F1F700002111F5CFA4
:104550002091E80025FF14C0EC0140E050E068E045
:1045600070E00E94A2248091E8008E778093E8009A
:1045700088E0FE01A3EAB2E001900D928A95E1F78E
:10458000DF91CF9108958093A0027093A20260936F
:10459000A1028091D602843001F582E08093E90087
:1045A0008FEF9091E800815095FD06C095ED9A95AA
:1045B000F1F700008111F5CF8091E80085FF0DC073
:1045C00040E050E063E070E080EA92E00E94A224C4
:1045D0008091E8008E778093E8000895BC0184E024
:1045E0000C94C322BC0183E00C94C3228091D502B9
:1045F000811109C00E9433260E9490268091E2001A
:1046000084608093E20008951092D50208950C947E
:104610007F216091D20281E0611101C080E00C94A1
:104620006A219091D60281E0943009F080E0609197
:10463000D2020C946F2142E061EC81E00E94AC2533
:1046400042E261EC82E00E94AC259091D60281E0CA
:10465000943009F080E06091D2020C94782180912E
:10466000D802833009F461C030F4813071F08230B7
:1046700009F49AC008958A3009F486C08B3009F491
:104680006CC0893009F0A8C020C08091D702813A5F
:1046900009F0A2C08091E800877F8093E8008091B4
:1046A000DB029091DC02892B21F468E083EA92E03E
:1046B00003C060E080E090E070E00E94ED24809113
:1046C000E8008B778093E80008958091D7028132CB
:1046D00009F082C08091DB029091DC02029708F021
:1046E0007BC08091E800877F8093E8008091E8009C
:1046F00082FD05C08091D6028111F8CF6DC0209156
:10470000F3008091F20090E0922B029731F48091B7
:10471000F100813011F0863021F48091F100809316
:10472000AB028091E8008B7753C08091D702813A29
:1047300009F052C08091DB029091DC02892B09F0D4
:104740004BC08091E800877F8093E8008091E8006B
:1047500080FFFCCF80914E0136C08091D70281321C
:10476000D9F58091DB029091DC02892BA9F580912B
:10477000E800877F8093E8000E94E1258091D902BC
:1047800080934E010C9433098091D702813221F538
:104790008091E800877F8093E8000E94E125809166
:1047A000DA028093AC0208958091D702813AA1F495
:1047B0008091E800877F8093E8008091E80080FF87
:1047C000FCCF8091AC028093F1008091E8008E775D
:1047D0008093E8000C94E125089584B7877F84BF17
:1047E0000FB6F894A895809160008861809360006E
:1047F000109260000FBE90E080E80FB6F8948093AE
:104800006100909361000FBE0C947A210E943326C0
:104810000E949026E2EEF0E08081846080837894AC
:104820000C94252982E491E00C94C4208091D60256
:104830008530A9F48091D602853079F40E94CB218D
:104840008091D4028823B1F30E948C21882391F3B4
:104850000E948C240E943309EDCF0C94F621089518
:1048600008950C943324292F332723303105C9F0C0
:1048700060F42130310581F02230310509F044C067
:104880008BE390E026E135E043C021323105E1F0D1
:104890002232310549F138C082E190E021E535E06E
:1048A00037C099278130910549F028F0029761F5CA
:1048B000E4EEF4E005C0E2E1F5E002C0E8EFF4E088
:1048C000849190E09F0124C06115710541F0613031
:1048D0007105D1F489E090E021E435E019C089E068
:1048E00090E028E235E014C06115710541F06130B7
:1048F000710551F48BE790E023E635E009C080E4D0
:1049000090E02EED35E004C080E090E020E030E063
:10491000FA0131832083089580E189BD82E189BD58
:1049200009B400FEFDCF8091D8008F7D8093D80020
:104930008091E00082608093E0008091E00081FD42
:10494000FCCF0895CF92DF92EF92FF920F931F93C7
:10495000CF93DF93EC018B017A010E940026811135
:1049600033C0E114F10439F0F70180819181081B13
:10497000190BC80FD91FC12CD12C0115110519F124
:104980008091E80085FD16C08091E8008E778093C5
:10499000E800E114F10449F0F70180819181C80E2B
:1049A000D91ED182C08285E00FC00E9400268823D4
:1049B00021F30AC089918093F10001501109FFEFA2
:1049C000CF1ADF0ADACF80E0DF91CF911F910F91EC
:1049D000FF90EF90DF90CF9008952091DD0230910D
:1049E000DE022617370748F06115710539F420916A
:1049F000E8002E772093E80001C0B901FC0120E017
:104A00006115710579F18091D6028823F1F1853025
:104A1000F1F18091E80083FD3CC08091E80082FDC7
:104A20002EC08091E80080FFEBCF2091F3008091B1
:104A3000F20090E0922B6115710551F088309105DC
:104A400038F421912093F100615071090196F3CF60
:104A500021E0089709F020E08091E8008E778093AC
:104A6000E800CECF2111CFCF0AC08091D602882393
:104A700061F0853061F08091E80083FD0AC080918B
:104A8000E80082FFF2CF80E0089582E0089583E09D
:104A9000089581E008952091DD023091DE0226170D
:104AA000370748F06115710539F42091E8002E7739
:104AB0002093E80001C0B901FC0120E061157105F7
:104AC00091F18091D602882309F440C0853009F421
:104AD0003FC08091E80083FD3DC08091E80082FDE9
:104AE0002FC08091E80080FFE9CF2091F3008091F2
:104AF000F20090E0922B6115710559F08830910514
:104B000040F424912093F10031966150710901968F
:104B1000F2CF21E0089709F020E08091E8008E773D
:104B20008093E800CBCF2111CCCF0AC08091D60270
:104B3000882361F0853061F08091E80083FD0AC030
:104B40008091E80082FFF2CF80E0089582E008952E
:104B500083E0089581E00895982F973068F5909349
:104B6000E900981739F07091EC002091ED00509118
:104B7000F00003C0242F762F50E021FD02C09F5F7C
:104B8000ECCF3091EB003E7F3093EB003091ED00A5
:104B90003D7F3093ED003091EB0031603093EB00BE
:104BA0007093EC002093ED005093F0002091EE0004
:104BB00027FDE5CF80E008958F708093E90081E0C4
:104BC00008958091D70287FF11C08091E80082FD8F
:104BD00005C08091D6028111F8CF11C08091E80004
:104BE0008B770BC08091D602882349F08091E80032
:104BF00080FFF8CF8091E8008E778093E8000895D9
:104C00002091E4003091E50095E64091EC00842F7E
:104C1000817040FF23C08091E80080FD1DC080911D
:104C2000D602882399F0853099F08091EB0085FDBC
:104C300011C04091E4005091E5002417350729F395
:104C4000915011F09A01E1CF84E0089582E0089537
:104C500083E0089581E0089580E008954091E800A0
:104C600042FFDDCF08950E94A1260E94A926E0EE12
:104C7000F0E0808181608083E8EDF0E080818F77D3
:104C8000808319BCA7EDB0E08C918E7F8C938081DE
:104C90008F7E80831092D50208950F931F93CF9338
:104CA000DF930E94A1260E94A926C8EDD0E088814A
:104CB0008F77888388818068888388818F7D8883C7
:104CC00019BC1092D6021092D2021092D402109205
:104CD000D30200EE10E0F80180818B7F8083888111
:104CE0008160888342E060E080E00E94AC25E1EED4
:104CF000F0E080818E7F8083E2EEF0E08081816051
:104D00008083808188608083F80180818E7F8083AA
:104D1000888180618883DF91CF911F910F910895E1
:104D2000E8EDF0E080818F7E8083E7EDF0E0808128
:104D30008160808384E082BF81E08093D5020C94FF
:104D40004D26E8EDF0E080818E7F80831092E200B6
:104D500008951092DA001092E10008951F920F92C8
:104D60000FB60F9211242F933F934F935F936F933E
:104D70007F938F939F93AF93BF93EF93FF93809114
:104D8000E10082FF0BC08091E20082FF07C08091AA
:104D9000E1008B7F8093E1000E9424298091DA005A
:104DA00080FF1FC08091D80080FF1BC08091DA0077
:104DB0008E7F8093DA008091D90080FF0DC080E162
:104DC00089BD82E189BD09B400FEFDCF81E08093F9
:104DD000D6020E94F62205C019BC1092D6020E948B
:104DE00004238091E10080FF19C08091E20080FFE0
:104DF00015C08091E2008E7F8093E2008091E200F6
:104E000080618093E2008091D80080628093D80016
:104E100019BC85E08093D6020E9409238091E100AD
:104E200084FF30C08091E20084FF2CC080E189BD06
:104E300082E189BD09B400FEFDCF8091D8008F7D4D
:104E40008093D8008091E1008F7E8093E100809173
:104E5000E2008F7E8093E2008091E2008160809387
:104E6000E2008091D202882311F084E007C0809193
:104E7000E30087FD02C081E001C083E08093D60299
:104E80000E9411238091E10083FF29C08091E200FC
:104E900083FF25C08091E100877F8093E10082E05D
:104EA0008093D6021092D2028091E1008E7F80938F
:104EB000E1008091E2008E7F8093E2008091E20029
:104EC00080618093E20042E060E080E00E94AC25D7
:104ED0008091F00088608093F0000E940723FF918A
:104EE000EF91BF91AF919F918F917F916F915F9162
:104EF0004F913F912F910F900FBE0F901F901895DB
:104F00001F920F920FB60F9211242F933F934F933E
:104F10005F936F937F938F939F93AF93BF93CF9341
:104F2000DF93EF93FF93C091E900CF708091EC0085
:104F3000D82FD17080FDD0E81092E9008091F00068
:104F4000877F8093F00078940E94C4271092E90034
:104F50008091F00088608093F000CD2BCF70C093DB
:104F6000E900FF91EF91DF91CF91BF91AF919F91B8
:104F70008F917F916F915F914F913F912F910F9002
:104F80000FBE0F901F9018951F93CF93DF93CDB74F
:104F9000DEB7AA970FB6F894DEBF0FBECDBFE7ED20
:104FA000F2E08091F100819322E0EF3DF207C9F732
:104FB0000E942F238091E80083FF2EC18091D702A9
:104FC0009091D802492F50E04A30510508F024C191
:104FD000FA01EE59FF4F0C946829803821F082388D
:104FE00009F01AC108C08091D3029091D40299238C
:104FF00089F082600FC08091DB028F70873008F0EB
:105000000BC18093E9008091EB0085FB882780F934
:105010001092E9009091E800977F9093E8008093C8
:10502000F1001092F100D1C0282F2D7F09F0F4C0BB
:10503000882319F0823061F0EFC08091D90281306D
:1050400009F0EAC0933009F080E08093D4022EC0CA
:105050008091D90281112AC08091DB028F702FEFDD
:10506000280F263008F0D8C08093E9002091EB008B
:1050700020FF1CC0933021F48091EB00806214C0AB
:105080009091EB0090619093EB0021E030E0A9015A
:1050900002C0440F551F8A95E2F74093EA00109230
:1050A000EA008091EB0088608093EB001092E900A9
:1050B0008091E800877F8093E8000E94E125ACC0E2
:1050C0008111AAC01091D9021F778091E3008078E6
:1050D000812B8093E3008091E800877F8093E80034
:1050E0000E94E1258091E80080FFFCCF8091E300E1
:1050F00080688093E300111102C082E001C083E068
:105100008093D60289C08058823008F085C0809193
:10511000D9029091DA028C3D53E0950779F583E04E
:105120008A838AE289834FB7F894DE01139620E0E0
:105130003EE051E2E32FF0E050935700E49120FF6E
:1051400003C0E295EF703F5FEF708E2F90E0EA3082
:1051500010F0C79601C0C0968D939D932F5F2431A8
:1051600049F74FBF8091E800877F8093E8006AE2AB
:1051700070E0CE0101960E94ED2416C06091DB0222
:105180007091DC02AE014F5F5F4F0E943124BC0181
:10519000892B09F441C09091E800977F9093E80033
:1051A00089819A810E944B258091E8008B778093BA
:1051B000E80032C0803881F58091E800877F8093D5
:1051C000E8008091D2028093F1008091E8008E7710
:1051D00072CF811121C08091D9029091DA02992772
:1051E0000297D4F48091E800877F8093E800809153
:1051F000D9028093D2020E94E1258091D2028111CE
:1052000006C08091E30087FD02C081E001C084E018
:105210008093D6020E941B238091E80083FF0AC07E
:105220008091E800877F8093E8008091EB008062A6
:105230008093EB00AA960FB6F894DEBF0FBECDBFE9
:10524000DF91CF911F9108950895CF938091D60259
:105250008823A1F0C091E900CF709091EC00892FD4
:10526000817090FD80E8C82B1092E9008091E800E1
:1052700083FD0E94C427CF70C093E900CF910895A9
:10528000AA1BBB1B51E107C0AA1FBB1FA617B7076C
:1052900010F0A61BB70B881F991F5A95A9F7809588
:1052A0009095BC01CD01089597FB072E16F400944C
:1052B00007D077FD09D00E94402907FC05D03EF4B5
:1052C000909581959F4F0895709561957F4F0895B2
:1052D000EE0FFF1F0590F491E02D0994FC01415061
:1052E000504030F001900616D1F73197CF01089564
:1052F000882799270895FB01DC0104C08D91019056
:10530000801921F441505040C8F7881B990B08952B
:10531000F999FECF92BD81BDF89A992780B508957D
:10532000A6E1B0E044E050E00C94C229A8E1B0E06E
:1053300042E050E00C94C229262FF999FECF92BD8D
:1053400081BDF89A019700B4021639F01FBA20BD4A
:105350000FB6F894FA9AF99A0FBE08950396272F7C
:105360000E949D290E949C29252F0E949D29242F5F
:105370000C949D290196272F0E949D290C949C290D
:10538000DC01CB01FC01F999FECF06C0F2BDE1BD05
:10539000F89A319600B40D9241505040B8F70895F4
:0453A000F894FFCFAF
:1053A40000000000490300000000000000000000AD
:1053B400000000000000211F321F421F00000000F7
:1053C400000000000000000000002C013400340242
:1053D4005502280850011E0A1401000200020201AD
:1053E400FFFF742297227822F222EE22772201E232
:1053F40000E900EA00B500B600B700CD008301CC97
:10540400008A01920194012102230224022502262A
:105414000227022A02B300B4006F00700081828365
:10542400E200E900EA00B500B600B700CD00830150
:10543400CC008A0192019401210223022402250254
:10544400260227022A02B300B4006F007000818292
:10545400836766363534979694959392919033F496
:10546400F7F6F500010202020200FF01000100004C
:0A547400FFFF0000010001FF00002F
:00000001FF
